:0200000089284D
:1000060083160313981809280000032883123F0853
:040016009900080045
:0E001A008312031322088A00210882000800C6
:1000280083120313F8010830FC00700DF80D7408F2
:10003800F80203182128F8070310F00DFC0B192803
:020048000800AE
:10004A000D208A110A128000840AA10A0319A20A41
:08005A00F003031D2528080036
:1000620083120313BD0103303D0203183F283D08EC
:100072003C07840020308000BD0A34283D083C073C
:1000820084008001BD033D083C07BE000A30F40035
:100092003B08F00014207808F0003030F0073E08EA
:1000A2008400700880000A30F4003B08F00014203D
:1000B2007008BB007008003A031D60286228BD0367
:0400C20044280800C6
:1000C60083120313BD013B0884000008BC003C08F2
:1000D600003A031978283C08BF000320BD0A3D08F2
:0C00E6003B0784000008BC006A280800EA
:1000F200831603139816903083129800831687177D
:10010200071383128C1E88281A08F0008228080020
:10011200013083120313AB000230AC000330AD0098
:100122000430AE000530AF000630B0000730B10039
:100132000830B2000930B3000A30B4001430B50000
:100142001E30B6002830B7003230B8003C30B9005B
:100152004630BA0033308316990018157920A00171
:100162002008083C031CBC2820082B3E8400000801
:10017200AA07A00AB128A0012008033C031CC82832
:100182002008343E84000008AA07A00ABD282A08D5
:10019200BB002330BC0031202330BB0063200B3076
:1001A200FB002630FC005D30FD00FD0BD628FC0B69
:0E01B200D628FB0BD62800000000DE28DF2830
:04400E00F22F000786
:00000001FF
